:020000040800F2
:1000000028010020D5000008430200084102000832
:1000100000000000000000000000000000000000E0
:10002000000000000000000000000000450500087E
:1000300000000000000000001D030008E1050008AA
:10004000E700000800000000E7000008E7000008E3
:10005000E7000008E7000008E7000008E7000008E4
:10006000E7000008E7000008E7000008E7000008D4
:10007000E7000008E70000084106000859060008EC
:1000800000000000E7000008000000000000000081
:1000900000000000E7000008E7000008E700000893
:1000A00000000000E700000800000000E700000872
:1000B0000000000000000000000000000000000040
:1000C0000348854600F02AF8004800472B0900083D
:1000D000280100200448804704480047FEE7FEE767
:1000E000FEE7FEE7FEE7FEE7E5050008C1000008C1
:1000F00030B50B46014600202022012409E00D46C0
:10010000D5409D4205D31D469540491B2546954047
:1001100040191546521E002DF1DC30BD064C01255C
:10012000064E05E0E36807CC2B430C3C984710349F
:10013000B442F7D3FFF7C8FF600900088009000840
:1001400038B50020074C034600900222402120468B
:1001500000F05CF803220621204600F047F800F08A
:1001600099F838BD00080048F0B500220124234664
:100170000D6893401D409D422BD10D79012D01D07A
:10018000022D13D1876855000326AE40B743876020
:100190004E79AE4085682E43866045689D43456034
:1001A00043688D799540ADB22B4343600668550096
:1001B0000323AB409E4306600E790768AE403E4382
:1001C0000660C6689E43C660CB79AB40C5682B43CA
:1001D000C360521C102ACAD30A7A002A026B09682B
:1001E00002D08A430263F0BD0A43FBE74B07DB0EF4
:1001F0009A40C90810B589000818016A0F249C406C
:10020000A1430162016A1143016210BDFFB583B0D1
:100210000F460F201C461546012140040C9E00F09D
:100220007FF86846009705718671C471012141719C
:100230000021017269460398FFF796FF07B0F0BDF1
:10024000FEE7704730B5837801210278002B15D086
:1002500094080E4BA400E41823689207D50EFF22E1
:10026000AA40934342789207120EAA401A43226092
:100270000078C006C00E8140054804E0D006C00EDC
:10028000814003488030016030BD000000E400E0A0
:1002900000E100E070B501218AB0C80200F04CF81E
:1002A000EF20079002206946088300240C844C83C9
:1002B00008A9194E8C7006A9304600F045FA602056
:1002C000694688800125CD80042008817F20039025
:1002D0000C824C8228028882CC8201A9304600F030
:1002E000F7F90821304600F027FA0121304600F0E6
:1002F000CDF90121304600F0D5F9012211463046F2
:1003000000F0DBF90E20694608704C708D7068466D
:10031000FFF798FF0AB070BD002C01407047000045
:10032000044A0029516901D0014300E08143516131
:100330007047000000100240044A0029916901D072
:10034000014300E0814391617047000000100240CA
:10035000F8B52C49044648680C222B4E104003D0B7
:10036000042801D00C281FD0264D26606868274934
:100370000006000F4000095A30460746FFF7B8FE56
:1003800060606968214A4905490F083A515CC840D4
:100390000546A0601E480169890F09D00169890FCF
:1003A00001290FD0680812E07D2080022060DBE781
:1003B0001448C030806A4000C10E1648891CFFF7FF
:1003C00097FE04E00069800F022801D0A808E060D1
:1003D0000C48016BC90601D4266100E02761016B5E
:1003E00089070AD0016B8907890F012907D0006BA3
:1003F000C043800700D16661F8BD6561F8BD6761E3
:10040000F8BD0000001002400048E8014009000863
:10041000002401400090D0030029016802D040224E
:10042000114301E0014A114001607047BFFF000025
:10043000F0B501210D0387B02846FFF77DFF0024AA
:10044000224E23460222102130460094FFF7DEFEA2
:1004500000230222082130460094FFF7D7FE1C4FEC
:1004600000230222102138460094FFF7CFFE02221B
:1004700004213046FFF7BAFE022203213046FFF77F
:10048000B5FE022204213846FFF7B0FE6846FF2180
:1004900084800531C1800721090201814481848162
:1004A000E910C18118210182448207218182094C0F
:1004B00001A9204600F010F82946204600F038F83F
:1004C00001212046FFF7A8FF07B0F0BD000C00484F
:1004D000000400480030014030B50268CC8993B276
:1004E000C122920113400A880D892243CC882C43F3
:1004F00022434C8922438C8922431A43026042687A
:10050000094B92B21A408B88134343600A8A0261F6
:100510000268042392B249889A4311430160C16979
:10052000024A1140C16130BDFFF00000FFF700003A
:100530004268034B1A40426042680A434260704777
:10054000FFEF0000704700003CB5002221480092F8
:10055000019201680123194301601E49C0318C6A70
:100560000F25ED02AC438C628C6A0725ED022C430B
:100570008C62194C022105680D400195009D6D1C8F
:100580000095019D002D02D1009DA542F3D1046884
:10059000A4071DD5114A01931368DB08DB00019302
:1005A0000B4313604168F02291430191416041681F
:1005B0000722120291430191416041688908890034
:1005C00041604168416041680907890FFBD13CBD2A
:1005D00001923CBD00100240FFFF000000200240DD
:1005E0007047000010B512480168012211430160F4
:1005F0004168104A11404160016B1322914301632D
:10060000002484600C49096A0A0C89B20A4209D1A3
:100610000268CA064905120E890E09020A430168DA
:1006200011430160FFF790FF0448446310BD0000D0
:10063000001002401CB8FFF800F8FF1F40200240E5
:1006400010B50448416B491C4163012100F01AF8C0
:1006500010BD0000002C014010B5084808220378A6
:100660000749002B02D08A61002101E08A62012142
:1006700001700121880700F005F810BD000000207E
:1006800000080048C94389B2016170470029016828
:1006900002D00122114301E0014A1140016070477C
:1006A000FEFF00000029416C03D00122D203114358
:1006B00001E04904490C41647047002AC26801D036
:1006C0000A4302E0C94389B20A40C2607047000091
:1006D00030B5026A154B1A400262026A93B2426850
:1006E000846992B2A4B27025AC43A5080C88AD0011
:1006F0002C430225AB438D891D434B882B430C4D66
:10070000A8420DD10825AB43CD891D4304239D4349
:100710008B882B43074D2A400D8A15434A8A2A436A
:100720004260846189684163036230BDFEFF00005E
:10073000002C0140FFFC00008269082392B29A431A
:100740000A4382617047000010B502680F4B92B2F5
:10075000984203D00124A407A04203D17024A243ED
:100760004C8822430A4CA04203D00A4C22400C89F8
:10077000224302604A68C2620A888262984201D1BA
:10078000897A01630121416110BD0000002C014004
:1007900000100040FFFC00000029016802D0012287
:1007A000114301E04908490001607047F0B5092094
:1007B0008BB001214004FFF7B3FD01218803FFF74F
:1007C000BBFD0927FF06012203213846FFF70EFD76
:1007D000012206211B48FFF709FD08200090022690
:1007E00069460E7101254D7100248C71CC7138461B
:1007F000FFF7BAFC4020009069460E711148FFF7E0
:10080000B3FCE120099440020594069407940490F7
:100810000C200D4C089004A9204600F02FF81B2056
:10082000694608734D738D7303A8FFF70BFD012212
:100830000649204600F00CF801212046FFF7ACFFE6
:100840000BB0F0BD000C0048003801400501050068
:1008500010B50B041C0E01238B40022C02D0032C7C
:1008600002D002E0001D00E008300168002A01D03B
:10087000194300E09943016010BD000030B5044603
:10088000006887B00D464008400020606068032182
:1008900009038843A9680143616020681849EA6830
:1008A0000840696811432A69024311432160A06826
:1008B00003210902884369690143A1606846FFF783
:1008C00047FD1048844201D1059800E00298216854
:1008D0000904296800D54000FFF70AFC2A6852087D
:1008E0008A4200D8401C2168090404D50107064A41
:1008F000490F1040084380B2E06007B030BD0000EF
:10090000F3E9FFFF00380140F0FF000002E008C8F3
:10091000121F08C1002AFAD170477047002001E079
:1009200001C1121F002AFBD17047FFF781FDFFF7BD
:100930003DFFFFF705FCFEE7000000000102030495
:10094000010006000100010001000100010001009A
:1009500002000400080010004000800000010002B6
:100960008009000800000020040000000C090008B5
:100970008409000804000020240100001C0900086C
:040980000000000073
:04000005080000C12E
:00000001FF
